:100000000C94E6000C940E010C940E010C940E015D
:100010000C940E010C940E010C940E010C940E0124
:100020000C940E010C940E010C9412040C94840494
:100030000C940E010C940E010C940E010C940E0104
:100040000C940E010C940E010C940E010C940E01F4
:100050000C940E010C940E010C940E010C94C1062C
:100060000C940E010C940E010C940E010C940E01D4
:100070000C940E010C940E010C940E010C940E01C4
:100080000C940E010C940E010C940E010C940E01B4
:100090000C940E010C940E010C940E010C940E01A4
:1000A0000C940E010C940E010C940E0136013901D2
:1000B00028012C0130015A015A015A013D01410128
:1000C00045014B014F015A01550100000000240079
:1000D00027002A002D003000080B00020202010058
:1000E000090400000102020000052400100105249B
:1000F000010101042402060524060001070581030D
:1001000010004009040100020A0000000705020275
:100110004000000705830240000004030904417207
:100120006475696E6F204C4C430041726475696E52
:100130006F204573706C6F72610012010002000045
:10014000004041233C800001010203011201000232
:10015000EF02014041233C80000101020301000045
:100160000000250028002B002E00310004040404A8
:10017000040304050202020204030202020206064C
:100180000606060604040202020404040802011022
:1001900040804010204080408008020401804020C0
:1001A00010020110801020404020000000020009D1
:1001B0000F0000030401000C00000000000000001C
:1001C000000000000000000000000B0711241FBE0B
:1001D000CFEFDAE0DEBFCDBF11E0A0E0B1E0E2E0BA
:1001E000F0E102C005900D92A432B107D9F721E0E9
:1001F000A4E2B1E001C01D92A439B207E1F710E01A
:10020000C6EED0E004C02197FE010E94F407C53E6F
:10021000D107C9F70E9420070C94FF070C94000037
:10022000E7EBF1E04491E8E9F1E02491E9E7F1E05E
:100230009491992309F451C04423E1F150E0FA016B
:100240003197EF30F105B0F5EA5AFF4F0C94F407FF
:10025000309180003F7707C0309180003F7D03C020
:1002600030918000377F3093800024C034B53F77D1
:1002700002C034B53F7D34BD1DC0309190003F7742
:1002800007C0309190003F7D03C030919000377FD0
:10029000309390000FC03091C0003F7703C0309181
:1002A000C0003F7D3093C00005C03091C200377F51
:1002B0003093C200E92FF0E0EE0FFF1FE25AFE4F2D
:1002C000A591B4919FB7F894EC91811103C020954A
:1002D0002E2301C02E2B2C939FBF0895FC018091EB
:1002E0009301811103C08FEF9FEF08959FB7F8949A
:1002F00082E08093E9002091F20030E012161306AC
:1003000014F421E030E02115310559F0289884E6F5
:10031000809392018091F10080838091F200882384
:1003200019F09FBFC90108958BE68093E800F9CFCB
:10033000CF92DF92EF92FF920F931F93CF93DF93B1
:100340006C017A018B01C0E0D0E0CE15DF0589F0A9
:10035000D8016D918D01D601ED91FC910190F08154
:10036000E02DC6010995892B11F47E0102C021966A
:10037000ECCFC701DF91CF911F910F91FF90EF90CC
:10038000DF90CF90089580918A0181110DC082E0A5
:100390008093860184E080938701109289011092F6
:1003A000880181E080938A0186E891E00895CF93E7
:1003B000DF931F92CDB7DEB76983DC01ED91FC912D
:1003C0000280F381E02D41E050E0BE016F5F7F4F7E
:1003D00009950F90DF91CF91089583E08093E90014
:1003E0008091F200882319F08AE38093E800089551
:1003F000CF93DF931F92CDB7DEB7FC01848595853F
:1004000097FD05C02FEF3FEF358724870BC0CE0146
:1004100001960E946E01019719F4898190E002C053
:100420008FEF9FEF0F90DF91CF9108950F931F9360
:10043000CF93DF931F92CDB7DEB78C01FC0184858B
:10044000958597FF0EC0CE0101960E946E0101971F
:1004500019F4298130E002C02FEF3FEFF801358712
:100460002487F801848595850F90DF91CF911F91A6
:100470000F910895FC018485958597FD0BC09FB76A
:10048000F89482E08093E9008091F2009FBF90E0B1
:10049000019608959FB7F89482E08093E9008091D7
:1004A000F2009FBF90E008954091300150913101DA
:1004B00020912E0130912F0142175307B4F49091EF
:1004C000E8009570E1F39091E80092FD19C08093E7
:1004D000F100809130019091310101968F7399273D
:1004E000892B19F48EEF8093E80080913001909170
:1004F00031010196909331018093300181E008959C
:1005000080E00895CF92DF92EF92FF920F931F93B6
:10051000CF93DF931F92CDB7DEB7182F062FE42EAF
:10052000862F880F8E5F99830E94540283E00E9479
:100530005402F12EC12E9981D92E8C2D8F1980173E
:1005400098F4F601E7FE02C0849101C080810E9408
:100550005402182F80E00E9454028123FFEFCF1A2B
:10056000DF0A8111EACF01C081E00F90DF91CF91C6
:100570001F910F91FF90EF90DF90CF900895DF9241
:10058000EF92FF920F931F93CF93DF93D82E8A01A0
:100590007B01E40EF51EEB01CE15DF0571F0D7FEF1
:1005A00003C0FE01849101C088810E9454022196FB
:1005B0008111F2CF8FEF9FEF01C0C801DF91CF9182
:1005C0001F910F91FF90EF90DF9008950F931F936D
:1005D000CF93DF931F92CDB7DEB782E0898342E4E9
:1005E00050E068ED70E080E80E94BF020E94C30105
:1005F000DC0112960D911C9113970115110569F0FC
:10060000D801ED91FC910280F381E02DBE016F5F76
:100610007F4FC801099597FF07C089810F90DF912F
:10062000CF911F910F910895F80100851185E5CFB5
:10063000615030F02091F100FC0120830196F8CF49
:10064000289884E68093920108953FB7F8948091AA
:10065000290190912A01A0912B01B0912C0126B57E
:10066000A89B05C02F3F19F00196A11DB11D3FBFEA
:10067000BA2FA92F982F8827820F911DA11DB11D78
:10068000BC01CD0142E0660F771F881F991F4A9574
:10069000D1F708958F929F92AF92BF92CF92DF923F
:1006A000EF92FF926B017C010E9425034B015C01DC
:1006B000C114D104E104F104F1F00E942503DC012E
:1006C000CB0188199909AA09BB09883E9340A10565
:1006D000B10570F321E0C21AD108E108F10888EEF3
:1006E000880E83E0981EA11CB11CC114D104E10442
:1006F000F10419F7DDCFFF90EF90DF90CF90BF901E
:10070000AF909F908F9008958F929F92AF92BF92DB
:10071000CF92DF92EF92FF920F931F93CF93DF93CD
:100720005C016B018A0180910B01882309F45EC092
:1007300080919301882309F459C08091350180FF8D
:1007400005C08091E00082608093E000E8018AEFBC
:10075000F82E93E0E92E2FE3822E3AE3932E209792
:1007600009F43DC08FB7F894E092E9009091E80059
:1007700095FF06C09091F200282D291B922F01C0F1
:1007800090E08FBF91110AC0FA94FF2079F161E0E7
:1007900070E080E090E00E944A03E1CF292F30E032
:1007A000C217D3070CF49C2F8FB7F894E092E9009E
:1007B0002091E80025FF11C0292F30E0C21BD30B88
:1007C000F601915020F041914093F100FACFC20E12
:1007D000D31E9091E80095FF13C08FBFC0CF5D98E6
:1007E00084E6809334011016110644F081E090E015
:1007F000F5019383828380E090E005C0C80103C0C7
:100800009092E800EACFDF91CF911F910F91FF9076
:10081000EF90DF90CF90BF90AF909F908F90089512
:100820000E94FA071F920F920FB60F9211248F9316
:100830009F938091E1009091E100937F9093E1007C
:1008400083FF0FC01092E90091E09093EB001092AB
:10085000EC0092E39093ED001092930198E0909356
:10086000F00082FF20C093E09093E9009091F200A5
:10087000992319F09AE39093E80090913401992319
:1008800039F090913401915090933401992389F17A
:1008900090919201992339F0909192019150909307
:1008A0009201992341F184FF10C08091E2008E7E75
:1008B00081608093E2008091E1008F7E8093E1006F
:1008C000809135018E7E806111C080FF16C08091BD
:1008D000E2008E7E80618093E2008091E1008E7E56
:1008E0008093E100809135018E7E81608093350197
:1008F00004C05D9ACDCF289AD6CF9F918F910F904B
:100900000FBE0F901F9018951F920F920FB60F9267
:100910001124CF92DF92EF92FF920F931F932F93A8
:100920003F934F935F936F937F938F939F93AF9377
:10093000BF93EF93FF93CF93DF93CDB7DEB76C9761
:10094000DEBFCDBF1092E9008091E80083FFFAC1BD
:1009500068E0CE0145960E94180382EF8093E8007C
:100960008D8987FF05C09091E80090FFFCCF03C000
:100970009EEF9093E800982F907609F0C6C09E896C
:100980002F89188D91110CC0803829F48091330182
:100990008093F10002C01092F1001092F10047C163
:1009A000422F50E0512B913051F4811140C1413020
:1009B000510509F03CC1809133018D7F0BC093300C
:1009C00061F4811134C14130510509F030C1809189
:1009D00033018260809333012AC1953041F48091C4
:1009E000E80080FFFCCF20682093E30020C1963010
:1009F00009F05FC0EB8CFC8C1092E9001092310181
:100A000010923001123091F510922F0110922E01A8
:100A10000E94E60299E0BE016F5F7F4FDB01E92F84
:100A20001D92EA95E9F799831A8391E09E8390EAF3
:100A300098879AEF99872091300130913101275F93
:100A40003F4F3C832B838D831092E900109231013C
:100A500010923001F0922F01E0922E0149E050E017
:100A600080E00E94BF020E94E602E1C0F0922F01E6
:100A7000E0922E010E94C301DC011296ED90FC90E1
:100A80001397E114F10409F4C0C0D701ED91FC9172
:100A90000480F581E02DBE016B5E7F4FC701099593
:100AA000009719F00CF0C3C0C6C0F701E084F184D0
:100AB000E8CF973009F4BFC0983021F481E08093EB
:100AC000F100B5C0993009F0B2C0837009F0B3C02D
:100AD000EDE0F1E081E021E036E39081992361F0DF
:100AE0008093E9002093EB0091919093EC00309378
:100AF000ED008F5F873089F78EE78093EA001092D0
:100B0000EA008F898093930192C08B8D9C8D109207
:100B1000E900109231011092300190932F018093DF
:100B20002E01898D811156C08E899D89913A59F483
:100B3000813209F080C047E050E064E071E080E07D
:100B40000E94BF0274C0913209F075C0833289F4EB
:100B5000888D90E0982F88272F89822BA0E0B0E025
:100B60008093000190930101A0930201B0930301CF
:100B70005EC0803269F48091E80082FFFCCF67E0BC
:100B800084E091E00E9418038BEF8093E80006C098
:100B9000823209F04CC08F8980930B018091320121
:100BA000882319F0EEEFFAE002C0E0E0F8E080916F
:100BB000040190910501A0910601B0910701803BCD
:100BC0009440A105B10509F088C080910B0180FF18
:100BD000A0C083C00E94C301DC0112960D911C913C
:100BE00013970115110539F1D801ED91FC91019090
:100BF000F081E02DBE016B5E7F4FC8010995811128
:100C000016C0F80100851185ECCF1130C1F013300A
:100C100091F48F89882309F455C08230E9F440E8C3
:100C20006FE08AE291E00E948202882321F08EEF39
:100C30008093E80087C081E28093EB0083C08B8DB6
:100C40009C8D089711F410932D0180912D01811135
:100C500036C06AE371E038C0813029F440E86BE0C7
:100C60008EE191E0E0CF833031F70E94C301DC01D7
:100C70001296ED90FC9013978E010F5F1F4F680145
:100C8000E114F10479F0D701ED91FC910680F78130
:100C9000E02DB801C7010995080F111DF701E08487
:100CA000F184EECFD8011C92F60101900020E9F703
:100CB0003197BF016C197D0940E0C601B4CF6CE4E7
:100CC00071E002C06AE171E06115710509F4B3CF0A
:100CD000FB01449150E080E833CF0FB6F894A8951B
:100CE00080916000886180936000109260000FBE68
:100CF000A895EE3F2AE0F20739F08091FE0A909124
:100D0000FF0A9183808393CF1092FF0A1092FE0A0C
:100D10008ECFEE3F8AE0F80731F080819181909389
:100D2000FF0A8093FE0A87E797E7918380839BE021
:100D300088E10FB6F894A895809360000FBE909359
:100D4000600075CF6C960FB6F894DEBF0FBECDBFB6
:100D5000DF91CF91FF91EF91BF91AF919F918F91D3
:100D60007F916F915F914F913F912F911F910F91C3
:100D7000FF90EF90DF90CF900F900FBE0F901F90DD
:100D800018951F920F920FB60F9211242F933F9335
:100D90008F939F93AF93BF938091250190912601EC
:100DA000A0912701B09128013091240123E0230F65
:100DB0002D3720F40196A11DB11D05C026E8230F93
:100DC0000296A11DB11D20932401809325019093CB
:100DD0002601A0932701B0932801809129019091C9
:100DE0002A01A0912B01B0912C010196A11DB11DEA
:100DF0008093290190932A01A0932B01B0932C0199
:100E0000BF91AF919F918F913F912F910F900FBE06
:100E10000F901F901895E6E3F1E01382128288EE9E
:100E200093E0A0E0B0E084839583A683B78387E155
:100E300091E0918380838FEF9FEF9587848708955A
:100E4000789484B5826084BD84B5816084BD85B5A5
:100E5000826085BD85B5816085BD80916E008160B1
:100E600080936E0010928100809181008260809357
:100E70008100809181008160809381008091800059
:100E800081608093800080919100826080939100C6
:100E900080919100816080939100809190008160A9
:100EA000809390008091C10084608093C100809104
:100EB000C10082608093C1008091C10081608093F5
:100EC000C1008091C30081608093C3008091C00005
:100ED00082608093C0008091C20081608093C200D4
:100EE00080917A00846080937A0080917A00826099
:100EF00080937A0080917A00816080937A0080915B
:100F00007A00806880937A001092930110923301E6
:100F1000109235018091D70081608093D70080EADC
:100F20008093D80089B5806189BD89B5826089BD0B
:100F300009B400FEFDCF61E070E080E090E00E9427
:100F40004A038091D8008F7C80618093D800809183
:100F5000E000807F8093E0008091E1008E7E8093AE
:100F6000E1008DE08093E200559A209AEEEFFFE7D2
:100F7000859194918B3F9C4D19F481E080933201CF
:100F8000E8E9F1E02491E9E7F1E08491882399F020
:100F900090E0880F991FFC01E653FF4FA591B49193
:100FA000FC01E25AFE4F859194918FB7F894EC9131
:100FB000E22BEC938FBFC0E0D0E081E00E941001F3
:100FC00068EE73E080E090E00E944A0380E00E94B7
:100FD000100168EE73E080E090E00E944A032097E1
:100FE00061F30E940000E9CFEE0FFF1F0590F4911E
:100FF000E02D099481E090E0F8940C94FF07F894B8
:02100000FFCF20
:10100200FFFFFFFF00E100000000000000C180813F
:1010120000000000000000D70184033A02F8011624
:0410220002ED0100DA
:00000001FF
